S020000064656D6F70726F675F6F6C696D6578696E6F5F73746D33322E737265635C
S3150800800000500020398300081D8300081F830008DC
S315080080102183000823830008258300080000000048
S315080080200000000000000000000000002783000890
S3150800803029830008000000002B8300082D83000810
S3150800804089830008898300088983000889830008D2
S3150800805089830008898300088983000889830008C2
S3150800806089830008898300088983000889830008B2
S3150800807089830008898300088983000889830008A2
S315080080808983000889830008898300088983000892
S315080080908983000889830008898300088983000882
S315080080A08983000889830008898300088983000872
S315080080B08983000889830008898300088983000862
S315080080C08983000889830008898300088983000852
S315080080D08983000889830008898300088983000842
S315080080E08983000889830008898300080000000046
S315080080F00000000000000000000000000000000072
S3150800810000000000000000005FF808F1EE11AA5513
S3150800811010B5054C237833B9044B13B10448AFF3B3
S3150800812000800123237010BD0C0000200000000011
S31508008130188D000808B5034B1BB103490348AFF374
S31508008140008008BD0000000010000020188D0008FF
S3150800815008B500F03DF800F00BF800F007F808BD88
S3150800816008B500F00FF800F002F808BD7047704730
S3150800817008B500222021024800F09AFA08BD00BF7F
S315080081800008014010B500F024F80E4B1B68C31A0E
S31508008190B3F5FA7F0CD304460B4B1B784BB9012277
S315080081A0094B1A702021094800F082FA054B1C6019
S315080081B010BD0022044B1A702021044800F078FAFA
S315080081C0F4E700BF2C00002028000020000801402A
S315080081D0704708B500F01EF908BD0000014A024BB9
S315080081E09A6070470080000800ED00E030B589B05D
S315080081F000240494059406940794174B9A6942F050
S3150800820020029A619A6902F020020192019A9A69FB
S3150800821042F004029A619A6902F004020292029AF2
S315080082209A6942F008029A619B6903F0080303936E
S31508008230039B0A4D22462021284600F039FA2023BE
S3150800824004930123059306940223079304A9284659
S3150800825000F042F909B030BD0010024000080140A4
S3150800826030B591B00024089409940B940C940194A9
S315080082700294039404940594012206924FF48033E1
S3150800828007930A9202250D950E934FF4E0130F9368
S3150800829006A800F029FA0F230193029503944FF4D8
S315080082A0806304930594294601A800F05DFC11B08B
S315080082B030BD08B5FFF792FF00F08EF8FFF7D0FF44
S315080082C0FFF794FFFFF744FFFFF74AFFFCE70000BC
S315080082D082B0104B9A6942F001029A619A6902F0DB
S315080082E001020092009ADA6942F08052DA61DB698B
S315080082F003F080530193019B074A536823F0E06318
S3150800830043F080635360536823F0E063536002B020
S31508008310704700BF00100240000001407047FEE7AA
S31508008320FEE7FEE7FEE770477047704708B500F0BE
S3150800833065F808BD70470000DFF834D0002103E077
S315080083400C4B5B58435004310B480C4B42189A426D
S31508008350F6D30B4A02E0002342F8043B094B9A4243
S31508008360F9D3FFF7E7FF00F0B3FCFFF7A2FF70476A
S31508008370005000205C8D0008000000200C00002042
S315080083800C00002034000020FEE7000010B504466B
S315080083900E4B18784FF47A73B3FBF0F30C4A106857
S315080083A0B0FBF3F000F082F868B90F2C01D9012070
S315080083B00AE0002221464FF0FF3000F043F8054B53
S315080083C01C60002000E0012010BD00BF0400002052
S315080083D0000000200800002008B5074A136843F08B
S315080083E010031360032000F01BF80020FFF7CEFFF0
S315080083F0FFF76EFF002008BD00200240034A1168FF
S31508008400034B1B780B441360704700BF30000020F5
S3150800841004000020014B1868704700BF3000002098
S31508008420074AD36823F4E0631B041B0C000200F41C
S31508008430E060184340F0BF6040F40030D0607047F9
S3150800844000ED00E030B4174BDB68C3F30223C3F139
S315080084500704042C28BF04241D1D062D18D9033B28
S315080084604FF0FF3505FA04F421EA0401994005FAAC
S3150800847003F322EA0303194300280BDB0901C9B2F7
S3150800848000F1604000F5614080F8001330BC704789
S315080084900023E5E700F00F000901C9B2024B1954A1
S315080084A0F4E700BF00ED00E014ED00E00138B0F19C
S315080084B0807F0AD2064B5860064AF02182F82310BC
S315080084C00020986007221A6070470120704700BF95
S315080084D010E000E000ED00E0F0B482B0002632467D
S315080084E0A2E0002D5AD0012D00D1CE68FF2B69D805
S315080084F08446FF2B69D89500DCF800400F27AF406B
S3150800850024EA070406FA05F52C43CCF800404C6823
S3150800851014F0805F00F087805F4CA56945F001057F
S31508008520A561A46904F001040194019C9508AF1C97
S315080085305A4C54F8274002F00307BF004FF00F0CBF
S315080085400CFA07FC24EA0C0C554CA04243D004F55F
S315080085508064A04200F0818004F58064A0427ED049
S3150800856004F58064A04234D0042435E04D4FBD4262
S3150800857014D00BD94C4FBD4210D007F58037BD42F9
S315080085800CD0A7F58017BD42B0D107E0A7F5801734
S31508008590BD4203D007F58037BD42A7D18D687DB1AE
S315080085A0012D08D044610826A0E7CE6808369DE765
S315080085B0CE680C369AE70461082697E7002695E701
S315080085C0042693E700F1040C93E7A2F10805AD0031
S315080085D092E7032400E00024BC4044EA0C04023578
S315080085E02E4F47F825404C6814F4803F39D02F4D5C
S315080085F02C681C432C604C6814F4003F37D02B4D74
S315080086006C681C436C604C6814F4801F35D0274D89
S31508008610AC681C43AC604C6814F4001F33D0234D7F
S31508008620EC682343EB6001320B6833FA02F430D06E
S315080086300124944023409C42F5D14D68122DB7D0B1
S3150800864094D8022DB1D07FF64CAF032DB6D0112D9C
S315080086507FF44CAFCE68043648E70124BCE7022411
S31508008660BAE7124D2C6824EA03042C60C3E70F4DC1
S315080086706C6824EA03046C60C5E70C4DAC6824EA10
S315080086800304AC60C7E7094DEC6824EA0303EB6012
S31508008690C9E702B0F0BC7047001002400000014074
S315080086A000080140000021100000311000040140BC
S315080086B012B90904016170470161704782B0084B1D
S315080086C01B68084AA2FB03235B0A00FB03F0019020
S315080086D000BF019B5A1E0192002BF9D102B07047C8
S315080086E000000020D34D6210002800F0F58170B517
S315080086F082B00446036813F0010F2CD0AB4B5B68BD
S3150800870003F00C03042B1DD0A84B5B6803F00C0385
S31508008710082B12D06368B3F5803F41D0002B55D1A2
S3150800872003F1804303F504331A6822F480321A6091
S315080087301A6822F480221A6037E09C4B5B6813F4AF
S31508008740803FE7D0994B1B6813F4003F03D063685A
S31508008750002B00F0C381236813F0020F76D0934BE9
S315080087605B6813F00C0F5FD0904B5B6803F00C034B
S31508008770082B54D02369002B00F08A808C4B0122E9
S315080087801A60FFF747FE0546884B1B6813F0020F71
S3150800879075D1FFF73FFE401B0228F5D90320A0E15B
S315080087A0824A136843F480331360636843B3FFF760
S315080087B031FE05467D4B1B6813F4003FCBD1FFF70E
S315080087C029FE401B6428F5D903208AE1B3F5A02FBA
S315080087D009D0764B1A6822F480321A601A6822F495
S315080087E080221A60E1E703F18043A3F53C331A6857
S315080087F042F480221A601A6842F480321A60D4E77A
S31508008800FFF708FE0546694B1B6813F4003FA2D024
S31508008810FFF700FE401B6428F5D9032061E1634B8E
S315080088205B6813F4803FA5D1604B1B6813F0020FF9
S3150800883004D02369012B01D0012052E15B4A136859
S3150800884023F0F803616943EAC1031360236813F050
S31508008850080F32D0A369002B5BD0564B01221A6051
S31508008860FFF7D8FD0546514B5B6A13F0020F21D17D
S31508008870FFF7D0FD401B0228F5D9032031E14B4A0A
S31508008880136823F0F803616943EAC1031360DDE75F
S31508008890474B00221A60FFF7BDFD0546434B1B6890
S315080088A013F0020FD2D0FFF7B5FD401B0228F5D909
S315080088B0032016E10120FFF701FF236813F0040FD8
S315080088C000F09880394BDB6913F0805F33D1374B62
S315080088D0DA6942F08052DA61DB6903F0805301936A
S315080088E0019B0125344B1B6813F4807F25D0E36870
S315080088F0012B36D0002B4CD103F1804303F504330A
S315080089001A6A22F001021A621A6A22F004021A622C
S315080089102CE0284B00221A60FFF77CFD0546234B06
S315080089205B6A13F0020FC8D0FFF774FD401B0228DC
S31508008930F5D90320D5E00025D4E71F4A136843F488
S3150800894080731360FFF766FD06461B4B1B6813F41E
S31508008950807FCCD1FFF75EFD801B6428F5D9032004
S31508008960BFE0124A136A43F001031362E3687BB35C
S31508008970FFF750FD06460D4B1B6A13F0020F38D160
S31508008980FFF748FD801B41F288339842F3D903204C
S31508008990A7E0052B12D0054B1A6A22F001021A62CB
S315080089A01A6A22F004021A62E0E700BF00100240C9
S315080089B00000424280044242007000404C4B1A6A52
S315080089C042F004021A621A6A42F001021A62CDE7FC
S315080089D0FFF720FD0646464B1B6A13F0020F08D028
S315080089E0FFF718FD801B41F288339842F3D903201C
S315080089F077E0E5B9E369002B72D03D4A526802F088
S31508008A000C02082A56D0022B17D03A4B00221A60BD
S31508008A10FFF700FD0446364B1B6813F0007F47D06E
S31508008A20FFF7F8FC001B0228F5D9032059E0304A65
S31508008A30D36923F08053D361DCE72E4B00221A60FA
S31508008A40FFF7E8FC05462A4B1B6813F0007F06D0A3
S31508008A50FFF7E0FC401B0228F5D9032041E0236A12
S31508008A60B3F5803F1AD022494B6823F47413226A5F
S31508008A70606A024313434B601E4B01221A60FFF7DC
S31508008A80C9FC04461A4B1B6813F0007F0ED1FFF78A
S31508008A90C1FC001B0228F5D9032022E0144A5368BA
S31508008AA023F40033A1680B435360DCE7002018E089
S31508008AB0002016E0012B16D00D4B5B6803F48031BD
S31508008AC0226A914201D001200BE003F47013626A16
S31508008AD093420AD0012004E001207047012000E0FB
S31508008AE0002002B070BD0120FBE70020F9E700BFB7
S31508008AF0001002406000424210B487B0164C94E859
S31508008B000F000DF1180C0CE90F00238AADF804309C
S31508008B10124B5B6803F00C02082A1AD1C3F383428E
S31508008B20624412F8102C13F4803F05D10C4800FB60
S31508008B3002F007B010BC7047084B5B68C3F34043AC
S31508008B40634413F8143C074800FB02F0B0FBF3F04B
S31508008B50EFE70448EDE700BF308D0008001002403B
S31508008B6000093D0000127A00002800F0A38070B5C5
S31508008B700446524B1B6803F007038B420CD24F4A3C
S31508008B80136823F007030B431360136803F0070306
S31508008B908B4201D0012070BD236813F0020F17D055
S31508008BA013F0040F04D0464A536843F4E063536055
S31508008BB0236813F0080F04D0414A536843F46053FE
S31508008BC053603F4A536823F0F003A0680343536099
S31508008BD00D46236813F0010F31D06368012B20D0AE
S31508008BE0022B25D0364A126812F0020F64D0344997
S31508008BF04A6822F0030213434B60FFF70BFC064654
S31508008C002F4B5B6803F00C036268B3EB820F16D038
S31508008C10FFF700FC801B41F288339842F0D9032005
S31508008C20B9E7274A126812F4003FE0D10120B2E7FB
S31508008C30234A126812F0007FD9D10120ABE71F4BF7
S31508008C401B6803F00703AB420CD91C4A136823F0D0
S31508008C5007032B431360136803F00703AB4201D0E5
S31508008C60012098E7236813F0040F06D0144A5368C6
S31508008C7023F4E063E1680B435360236813F0080F9D
S31508008C8007D00F4A536823F46053216943EAC103A6
S31508008C905360FFF731FF0A4B5B68C3F30313094AB6
S31508008CA0D35CD840084B1860084B1868FFF76EFB72
S31508008CB0002070E70120704701206CE70020024081
S31508008CC000100240448D0008000000200800002023
S31508008CD070B500250C4E0D4CA41BA410A54209D155
S31508008CE000F01AF800250A4E0A4CA41BA410A54247
S31508008CF005D170BD56F8253098470135EEE756F888
S31508008D00253098470135F2E7548D0008548D000840
S31508008D10548D0008588D0008F8B500BFF8BC08BC8B
S31508008D209E467047F8B500BFF8BC08BC9E4670471B
S31508008D3002030405060708090A0B0C0D0E0F10108E
S31508008D400102000000000000000000000102030408
S30908008D5006070809F3
S30908008D54358100084F
S30908008D58118100086F
S31108008D5C0024F4000100000010000000D4
S7050800833936
